:10000000830100308A003B28F10003088301A60029
:100010007008A700831203138C1C30288C10A00AD0
:100020000319A10AA20A0319A30A2108803AF000C1
:1000300083307002E93003192002031C23280130A9
:100040008606A001A1012308803AF000AE307002BC
:10005000E13003192202031C302886140615861588
:1000600083168C14031383122708F00026088300DC
:10007000F10E710E090020308400263044208301E7
:10008000EB2F04068001840A04060319003441287A
:100FB2008312031312179216121692159214121418
:100FC20014308316920083128C1083168C148312B1
:100FD20012150800D9270B178B1706108316061057
:100FE2008312861006118611831686100611861149
:0E0FF2008312A001A101A201A3016400FE2F41
:02400E00463F2B
:00000001FF
